:020000000C945E
:1000020065000C9400000C9400000C9400000C9409
:1000120000000C9400000C9400000C9400000C945E
:1000220000000C9400000C9400000C9400000C944E
:1000320000000C9400000C9400000C9400000C943E
:10004200C7000C9400000C9494000C9400000C94D3
:1000520000000C9400000C9400000C9400000C941E
:1000620000000C9400001027E80364000A0001005D
:10007200001000011000010000000000000000005C
:10008200000000000000000000000000000000006E
:10009200000000000000000000000000000000005E
:1000A2000000000000000000000A0A0A0A0A0A0A08
:1000B2000A0A0A0A0A0A0A0A0A00010002007A0067
:1000C200020004007C000000F894EE27EFBBF1E090
:1000D200F5BFE5BF8DE0A2E0BB27ED938A95E9F776
:1000E20080E098E0A0E0B1E0ED930197E9F7ECEB56
:1000F200F0E085919591009761F0A591B5910590F9
:100102001590BF01F00105900D920197E1F7FB01F7
:10011200F0CFE8E0EEBBEFEFEDBFE8E0EEBFC0E00E
:10012200D3E00C941603AA93EA93FA93EFB7EA93F7
:100132001A930A931091C0000091C600E12FEC714E
:10014200E9F4E091BD03EF5FE093BD03E150F0E01D
:10015200EC55FC4F0083A091BD03A93119F4E0E0F6
:10016200E093BD03A091BF03AF5FA093BF03A9318A
:1001720029F4E0E0E093BF03689425F8099119910E
:10018200E991EFBFF991E991A99118950A921A9212
:100192006A937A938A939A93AA93BA93EA93FA9375
:1001A200EFB7EA93E0912603F09127033196E093AB
:1001B2002603F09327030E944417E1E5F1E00E9431
:1001C200631F0E2E0E944417E3EAF2E00E94631FAF
:1001D200E02909F499C1A0912403B0912503E4E137
:1001E200F0E00E94751F0E2EE0910603F0E0749776
:1001F2000E9449170E94691F0E22A0911503EEE08A
:100202000E94591FE02121F0E0911503EF5F03C026
:1002120024FC03C0E0E0E0931503A0911503AE3087
:1002220011F4689424F8E0912403E0930603A0916A
:100232001603A13029F4F79B02C0F79801C0F79A80
:10024200E1E02E26A0916803B091690380916A03D0
:1002520090916B030E944E17E0938C03F0938D03F1
:1002620060938E0370938F030E945517A0E7B3E04B
:100272000E945A170E946117ACE9B3E00E945A1714
:100282000E9466170E946F170E94941EE0937003EB
:10029200F09371036093720370937303A0919C03B4
:1002A200B0919D0380919E0390919F03E0E0F0E066
:1002B20060E772E40E94941EE0939C03F0939D0316
:1002C20060939E0370939F030E9474170E94791794
:1002D2000E2E0E947E170E947917E02161F1E091B3
:1002E2009C03F0919D0360919E0370919F030E9475
:1002F20066170E94941EE0939803F093990360930B
:100302009A0370939B030E948317AAE3B3E00E94AF
:100312008C17A0919803B091990380919A039091C0
:100322009B030E944E17E0937803F0937903609346
:100332007A0370937B030E949117E0E0F0E06AE792
:1003420074E40E949A170E949F170E94F61DE09380
:100352008003F093810360938203709383030E946E
:10036200A8170E94BB17ACE4B3E00E94C0170E941A
:10037200C5170E9491170E94BC1D0E949A17E09314
:100382009003F09391036093920370939303A0916F
:10039200A003B091A1038091A2039091A3030E94B4
:1003A200F61DE093A003F093A1036093A203709360
:1003B200A303A0911D03E5E20E94CE17AEE4B3E0D1
:1003C2000E94C0170E94DE17A0E0B0E080E89FE321
:1003D2000E94941EA0919003B09191038091920388
:1003E200909193030E94461EE0938803F093890341
:1003F20060938A0370938B030E94E717ABE1B3E02B
:100402000E94831DEC930E94DE170E94F0170E9447
:10041200F61D0E94F917E0917003F091710360914B
:100422007203709173030E9402180E94D91E68F52C
:10043200E0917803F091790360917A0370917B03E4
:100442000E9402180E94F61DE0937403F093750354
:1004520060937603709377030E9402180E940B1830
:100462000E94EF1DDF01CB010E9483170E94941EA0
:10047200A0E0B0E081E695E40E94461EA8E4B3E065
:100482000E94C017689423F802C0E8E02E260E945A
:10049200DE17A0917C03B0917D0380917E03909141
:1004A2007F030E94F61DE0937C03F0937D0360932B
:1004B2007E0370937F03AAE2B3E00E948C17ABE144
:1004C200B0E00E946A200E941418EA17FB0740F469
:1004D200E0912A03F0912B03ABE1B0E00E947A2075
:1004E2000E94F0170E946F170E94461EA8E2B3E016
:1004F2000E948C17A0911303AC3308F4F298A091D8
:100502001303AC3309F4F29A0E944417A33AE2E0CF
:10051200BE0709F061C0A09112030E9419180E943F
:100522001E180E9427180E947B1F0E942C1891F00F
:10053200E0911303EF5FE0931303E0911203F0E005
:100542003296A0911303B0E0EA17FB0719F4ECE32B
:10055200E0931303E0E0E0932603E0932703C394C0
:10056200A0913E03B0913F03E8E5F2E00E946F1FC5
:100572000E2E0E943418E02199F0E0913E03F09192
:100582003F033196E0933E03F0933F030E941E180F
:100592000E949D202CF4E0E0E0933E03E0933F03B1
:1005A200ECE3EC15C9F4CC24E0910003EF5FE09397
:1005B2000003A0910003AC3379F4E0E0E093000380
:1005C200E0910103EF5FE0930103A0910103A431E5
:1005D20019F4E0E0E0930103E991EFBFF991E991A9
:1005E200B991A991999189917991699119900990FB
:1005F2001895AA93E881E066E0937C0085E28A95EB
:10060200F1F7E0917A00E064E0937A00E0917A00F9
:10061200E071E1F3E0917A00E061E0937A00E09129
:100622007800F091790021960895EF978DE3A2E08A
:10063200B0E0EEE7F0E00E94B220FF2401E020E00B
:10064200E0E8E0936100E0E0E0936100EFE0E4B90C
:10065200E1E0E5B9E0E0E7B9E8B9EAEFEAB9E7EEE7
:10066200EBB9E0E0E4BDE3E0E5BDE0E0E6BDE7BD17
:10067200E8BDE1EAE0938000E2E0E0938100E0E09F
:10068200E0938500E0938400E0938700E093860086
:10069200E0938900E0938800E0938B00E0938A0066
:1006A200E093B600E1EAE093B000E2E0E093B1004B
:1006B200E0E0E093B200E093B300E093B400E1E045
:1006C200E0936E00E0E0E0936F00E0937000E0934F
:1006D2006900EDBBE0936800E093C000E8E9E093B5
:1006E200C100E6E0E093C200E0E0E093C500E7E489
:1006F200E093C400E0E8E0BFE0E0E0937F00E09335
:100702007E00E0E6E0937C00E7E2E0937A00E0E03E
:10071200E0937B00ECBDE093BC0078940E94391812
:100722000E944118EAE09E1650F4A3E2B0E0E0E035
:10073200F0E00E947A20ADE1B0E00E947A200E94AF
:100742004B180E9452180E945918E8ECF0E0E0930E
:100752004203F0934303EDE0E0930703A0E0B0E02F
:100762000E946E20E0930803A1E0B0E00E946E2098
:10077200E0930903A2E0B0E00E946E20E0930A0336
:10078200A3E0B0E00E946E20E0930C03A4E0B0E08E
:100792000E946E20EC8BA5E0B0E00E946E20ED8BF3
:1007A200A6E0B0E00E946E20EE8BA7E0B0E00E94CF
:1007B2006E20E0930D03A8E0B0E00E946E20E0936B
:1007C2000E03A9E0B0E00E946E20E0930F03F798B9
:1007D200F198AAE0B0E00E946E20E0931203A9E132
:1007E200B0E00E946A200E946018A4E1B0E00E947A
:1007F2006E20E88BA5E1B0E00E946E20E98BA6E1B5
:10080200B0E00E946E20EA8BABE0B0E00E946E2066
:10081200EC87ACE0B0E00E946E20ED87ADE0B0E086
:100822000E946E20EE87AFE1B0E00E946A20EB8367
:10083200FC83AEE0B0E00E946E20E0931703AFE0CD
:10084200B0E00E946E20E0931903A0E1B0E00E94A4
:100852006E20E0931803ABE1B0E00E946A20E093BF
:100862002A03F0932B03ACE7B3E00E945A17ADE1E1
:10087200B0E00E946A20ACE6B3E00E9465180E94D4
:100882000B18A8E2B3E00E948C170E94F0170E9496
:100892006F170E94941E0E94F917A1E1B0E00E9416
:1008A2006E203E2FA1E2B0E00E946A20EF83F8871B
:1008B200A2E1B0E00E946E20E88FA3E1B0E00E94C6
:1008C2006E20EF8BA3E2B0E00E946A20A0E8B3E0C2
:1008D2000E946518A5E2B0E00E946A200E946C188E
:1008E200A7E1B0E00E946E20E0931D03A8E1B0E012
:1008F2000E946E200E94AD2022F8A7E2B0E00E9482
:100902006A200E947118A0910303A43128F4E09197
:100912000303EF5FE0930303A0910303A43189F47F
:10092200E0E0E0931E03E0931F03EBE0E09320037B
:10093200E8EBE0932103E0E0E093BD03EAE0E0931B
:100942000303A091BD03AB30A9F4E091A703E093A8
:100952001E03E091A803E0931F03E091A903E09333
:100962002003E091AA03E0932103E0E0E093BD03BA
:10097200E0930303A091BD03AC30C0F0E0E0E0934C
:10098200A403E093A503E093A603E093A703E093F7
:10099200A8030E944B18E0E0E093AB03E093AC03A2
:1009A200E093AD03E093AE03E093BD03E8EC5E1683
:1009B20030F45394E4E1E51511F4E1E04E2E0E9487
:1009C2003918A0E00E9476183B97D8F0A0E00E9468
:1009D2007B18662777270E9482180E94C517A8EE07
:1009E200B3E080E090E00E94C61FDF01CB010E94CD
:1009F2008B18662777270E9408200E948218E894A5
:100A0200F3F80E9490180E944118E7EAE0937A00F6
:100A1200A2E00E947B18DF01E5E0F0E00E94CB1F1C
:100A2200BE2E0E949018A3E00E9476188E2E0E947D
:100A32009018A7E00E9476180E9497180E949018BA
:100A4200A5E00E9476181E2F0E949018A0E00E9436
:100A52007618DE2E0E949018A1E00E947618AE2E23
:100A62000E949018A6E00E947618EA87E7E2E093D7
:100A72007A00E1E0E51509F047C00E944917E2E378
:100A8200F0E00E94751F0E2E0E949C180E946F1F9C
:100A9200E02111F0E5E0E987A12FE2E30E945E1F69
:100AA2000E2EEAEF0E94591FE02111F0E6E0E987DD
:100AB2000E949C180E94751F0E2E0E94A018E02909
:100AC20011F0E7E0E987A12FEAEF0E945E1F0E2EE8
:100AD200EEE10E94591FE02911F0E8E0E987EAE01F
:100AE2008E1620F4EFEF8E2EECE00DC0EAE0AE168B
:100AF20020F4EFEFAE2EEEE006C0EAE0DE1620F4C0
:100B0200EFEFDE2EEFE0E9870E949C180E94751F2E
:100B12000E94A61839F0E1E0E987E8E2F0E00E94DD
:100B2200971807C00E94A0180E94A61811F0E2E0D0
:100B3200E987A12FEAEF0E945E1F0E94A61811F01A
:100B4200E3E008C0A12FEEE10E94591F0E94A618FF
:100B520019F0E4E0E9871CE3A9850E94B218A9858F
:100B6200E7E00E94451F0E2AE1E00E94451F0E2A7F
:100B7200E2E00E94451FE02929F0E12FF0E00E9407
:100B8200971818E2A9850E94B718A985E8E00E9483
:100B9200451FE02909F018E2A985AE3011F4EFEF04
:100BA200AE2EA985AF3011F4EFEFDE2EA985AC3061
:100BB20011F4EFEF8E2E0E94BC180E94591FE02103
:100BC20099F06894F3F8F39B04C0F398F49A02E066
:100BD2000BC0F49B04C0F498F59A03E005C0F59BA2
:100BE20003C0F598F39A01E00E944917D39708F4DD
:100BF20052C00E94CB180E94D018E02F0E94D71832
:100C020020F0E8ECF0E00E949718E02F0E94E7182D
:100C12000E94F718AC91A130E8F10E94FE180E94E0
:100C220007190E94A8204CF40E94F7180E94131979
:100C32000E94051F0E941E1923C00E9427190E94AC
:100C42002919EF930E9427190E943219AF91EA23C2
:100C520079F00E94F7180E9413190E940A1FA093AC
:100C62005003B0935103809352039093530308C0EF
:100C72000E9427190E943B191CF00E9445190AC0C4
:100C8200A0915003B091510380915203909153036C
:100C92000E944D1904C00E9454190E9445190E94D5
:100CA2005A190E9460190E220E946519E02139F03A
:100CB200E0912203E09314036894F0F821F80E9473
:100CC200CB18309721F4E0E0E093150306C0A09121
:100CD2001503A23010F4E89424F80E94CB18E09394
:100CE2002403F09325030E94CB18309719F4E8945B
:100CF20021F812C0A0E021FCA1E0E0E00E94451F23
:100D02000E2EA09114030E946C1931F0E0E0E093E2
:100D120014030E945419F198A0911403A13038F0E1
:100D2200F19AE0911403F0E00E94971801C0F19843
:100D3200E09105030E944917F0E0AE17BF0720F0CB
:100D4200E0912203E0930503E0910503F0E035977B
:100D52000E944917AE17BF0770F4E0912203E09397
:100D6200050324FE08C0E2E0E0931A03E89424F8A5
:100D7200E0E0E0931503A0911A030E9419180E9463
:100D820071190E948B1F0E22A09117030E947819DD
:100D92001E2EA0911A030E9419180E9471190E9416
:100DA200831F0E22A09118030E947819E12959F09D
:100DB2000E9449171B9710F00E945419E0911A03E0
:100DC200E150E0931A030E947D190E94831F0E9442
:100DD2008A190E9494190E948B1FE02161F10E94DE
:100DE20099190E94A119A4F0A0915C03B0915D032E
:100DF200EB81FC81EA1BFB0BA3E0B0E00E94C11F68
:100E02000E94A919AE1BBF0BA0934403B0934503E4
:100E12000E9499190E949D202CF40E94AE193397CA
:100E22000E94B319A0914503AA232AF4E0E0E093BB
:100E32004403E09345030E947D190E94A32074F5A8
:100E42000E947D190E940A1F0E94A11974F0AB81B1
:100E5200BC81E0915C03F0915D03EA1BFB0B0E94F5
:100E6200A919EA0FFB1F0E94B3190E947D190E9463
:100E72000A1FA230E0E0BE07E0E08E07E0E09E0736
:100E82002CF00E94AE1931960E94B3190E94A91942
:100E9200A93CE0E0BE0714F00E9452180E94AE196D
:100EA2000E944917EA17FB0720F40E94AE190E941C
:100EB20097180E94B81909F008F42DC00E94C919A8
:100EC200DF01CB01E0E0F0E060EA70E40E94D91EAD
:100ED20009F008F40CC00E94C919A0E0B0E080E457
:100EE20090E40E94461E0E94D8190E94E1190E94B5
:100EF200C9190E94932034F40E94C9190E94D8197A
:100F02000E94E119A0914703AA232AF4E0E0E093AA
:100F12004603E09347030E94B81930F50E94E61990
:100F2200DF01CB01E0E0F0E060E470E40E94D91E52
:100F320009F008F405C00E94F5193A960E94E119D9
:100F42000E94E6190E9493202CF40E94F519339610
:100F52000E94E119A0914603B0914703A13DE7E049
:100F6200BE0714F00E9459180E944917EAE00E9435
:100F7200BB1FDF010E94F519EA17FB0740F4A0919D
:100F82004603B09147030E94FA190E949718E09114
:100F92002203EA8F1333A0F0E0E0E0931403E12F81
:100FA200F0E0F2970E943B1F0E94BC1DA6EFB8E240
:100FB2008CE99FE30E94461E0E94831D1E2F01C0E2
:100FC20010E0AB2DE4E60E94591F0E2EA0E0F0992E
:100FD200A1E0E1E00E94451F0E942C181E2E0E94F3
:100FE200FF19A0913E03B0913F030E94631F0E942C
:100FF200041A0E943418E021E129B9F0E091280393
:10100200F0912903ADE1B0E00E947A200E940C1A0F
:101012000E94681AA4E6B0E00E944C1D5F98A8EEF8
:10102200B3E00E944C1D0C943817E0910E03E0933C
:10103200B300AA2DEAE00E945E1F0E2E0E946019E4
:10104200E02111F0E894F2F8AA2DE8E60E94C51A10
:101052000E946019E02171F06894F2F8E0911603A1
:10106200EF5FE0931603A0911603A33019F4E0E0BA
:10107200E0931603E0911603E03029F4E0E0E093F8
:10108200B400F7980FC0A0911603A13019F4E091B3
:101092000F0306C0A0911603A23021F4F79AEFEFD6
:1010A200E093B4000E9449170E9479170E2EA12FD7
:1010B200E0E00E945E1F0E22A09116030E946C19AE
:1010C200F9F0E0910403EF5FE0930403A0910403BD
:1010D200E5E00E945E1F0E2EE4E10E94591FE0210E
:1010E20041F0E0910403E170AFEFEA02F001E09316
:1010F200B400A0910403A03118F0E0E0E0930403EF
:10110200EAE0E81510F4E894F1F80E94D01A0E947F
:10111200D61A0E946019E02131F06894F1F82F5F2D
:10112200283009F420E00E94D01AA0911103EFEFB9
:101132000E94591FE02121F0E0911103EF5F03C0EB
:10114200E894F1F8E0E0E0931103A0911103A431D7
:10115200A9F4AA81E0E00E94541F0E2E0E94601999
:10116200E02119F0EA81E150EA83233610F423E604
:1011720005C020E00E940C1A0E94681A0E94D01A30
:101182000E94D61AAA81E4E60E944F1F0E94DE1A2C
:1011920051F06894F1F8EA81EF5FEA83AA81A436FC
:1011A20011F4E0E0EA83EAE0E91510F4E894F0F8DB
:1011B2000E945A190E9465190E22AA81E0E00E943B
:1011C2004A1F0E94DE1A51F06894F0F8EA81E15059
:1011D200EA83AA81AF3F11F4E3E6EA83EAE0ED1580
:1011E20010F4E894F3F80E94BC180E94451FE02115
:1011F20009F47EC16894F3F8AA81A13049F4A09160
:101202000803A13028F4E0910803EF5FE09308039C
:10121200AA81A23049F4A0910903A23328F4E091F3
:101222000903EB5FE0930903AA81A33049F4A0917B
:101232000A03A43628F4E0910A03EE5FE0930A035E
:10124200AA81A43049F4A0910C03A83228F4E091B9
:101252000C03EF5FE0930C03AA81A53031F4AC8953
:10126200A43618F4EC89EF5FEC8BAA81A63031F436
:10127200AD89A43618F4ED89EF5FED8BAA81A73012
:1012820031F4AE89A43618F4EE89EF5FEE8BAA81B1
:10129200A83049F4A0910D03A13028F4E0910D0388
:1012A200EF5FE0930D03AA81AD3069F4A0912C03A6
:1012B200B0912D03A433E8E0BE0728F40E948B18F6
:1012C20031960E946018AA81AE3031F4A889A43602
:1012D20018F4E889EB5FE88BAA81AF3031F4A98971
:1012E200A43618F4E989EB5FE98BAA81A03131F4C5
:1012F200AA89A43618F4EA89EB5FEA8BAA81A131A4
:1013020031F4AC85A83C18F4EC85EB5FEC87AA813C
:10131200A23131F4AD85A83C18F4ED85EB5FED8781
:10132200AA81A33131F4AE85A83C18F4EE85EB5FB7
:10133200EE87AA81A43169F4A0913C03B0913D03E8
:10134200A835E2E0BE0728F40E94FF197E960E94AB
:101352007118AA81A53159F4AB81BC81A33AE1E0AD
:10136200BE0728F4EB81FC813196EB83FC83AA81D2
:10137200A63149F4A0911703A13028F4E091170394
:10138200EF5FE0931703AA81A73149F4A0911903F3
:10139200A23328F4E0911903EF5FE0931903AA81C5
:1013A200A83149F4A0911803A13028F4E091180360
:1013B200EF5FE0931803AA81A93119F43F3008F4D2
:1013C2003F5FAA81AA3159F40E94E51AAC3BE2E0E0
:1013D200BE0728F40E94EA1A31960E946C18AA816C
:1013E200AB3149F4A0911D03AA3F28F4E0911D03FB
:1013F200EF5FE0931D03AA81AC3161F4A0E022FC0F
:10140200A1E0A13038F4E0E022FCE1E0EF5F0E94CD
:10141200AD2022F8AA81AD3169F40E947417A43F6D
:10142200E1E0BE0738F40E9455173A96E093340380
:10143200F0933503AA81AE3169F40E947E17A83574
:10144200E2E0BE0738F40E9461173A96E093400347
:10145200F0934103AA81AD3531F4A98DA73018F478
:10146200E98DEF5FE98FAA81AE3561F4AF81B8856E
:10147200A031E7E2BE0730F4EF81F885EC59FF4F67
:10148200EF83F887AA81AF3531F4A88DA83C18F410
:10149200E88DE65FE88FAA81A03631F4AF89A233E6
:1014A20018F4EF89EF5FEF8BAA81A13649F4A0917E
:1014B2001203AC3328F4E0911203EF5FE0931203BE
:1014C200AA81A23649F4A0910F03AA3F28F4E09121
:1014D2000F03E65FE0930F03AA81A33649F4A091BC
:1014E2000E03AA3F28F4E0910E03E65FE0930E0399
:1014F200EAE0EA1510F4E894F2F8AA2DEAE00E9474
:10150200C51AA22FE3E60E94451FE02109F47DC11E
:101512006894F2F8AA81A13049F4A0910803A1309D
:1015220028F0E0910803E150E0930803AA81A23079
:1015320049F4A0910903AB3028F0E0910903E5508A
:10154200E0930903AA81A33049F4A0910A03AD33C1
:1015520028F0E0910A03E250E0930A03AA81A43042
:1015620049F4A0910C03A53128F0E0910C03E1505D
:10157200E0930C03AA81A53031F4AC89A13018F0B4
:10158200EC89E150EC8BAA81A63031F4AD89A1300F
:1015920018F0ED89E150ED8BAA81A73031F4AE89C4
:1015A200A13018F0EE89E150EE8BAA81A83049F4FF
:1015B200A0910D03A13028F0E0910D03E150E093DA
:1015C2000D03AA81AD3069F4A0912C03B0912D03D3
:1015D200AD36E7E0BE0728F00E948B1831970E94D3
:1015E2006018AA81AE3031F4A889A63018F0E889D3
:1015F200E550E88BAA81AF3031F4A989A63018F002
:10160200E989E550E98BAA81A03131F4AA89A63093
:1016120018F0EA89E550EA8BAA81A13131F4AC8550
:10162200A13018F0EC85E550EC87AA81A23131F4A3
:10163200AD85A13018F0ED85E550ED87AA81A33183
:1016420031F4AE85A13018F0EE85E550EE87AA811F
:10165200A43161F4A0913C03B0913D030E94992012
:1016620028F40E94FF197E970E947118AA81A53161
:1016720059F4AB81BC81A332E1E0BE0728F0EB81D3
:10168200FC813197EB83FC83AA81A63149F4A091B6
:101692001703A13028F0E0911703E150E0931703FC
:1016A200AA81A73149F4A0911903A23028F0E09150
:1016B2001903E150E0931903AA81A83149F4A091DA
:1016C2001803A13028F0E0911803E150E0931803C9
:1016D200AA81A93119F4323008F03150AA81AA3115
:1016E20059F40E94E51AA935E2E0BE0728F00E94EB
:1016F200EA1A31970E946C18AA81AB3149F4A09181
:101702001D03A23028F0E0911D03E150E0931D0378
:10171200AA81AC3179F4A0E022FCA1E0A13050F022
:10172200A0E022FCA1E0E1E00E946620EA1B0E9408
:10173200AD2022F8AA81AD3161F40E9474170E9493
:10174200992038F40E9455173197E0933403F093AF
:101752003503AA81AE3161F40E947E170E9499205E
:1017620038F40E9461173197E0934003F0934103EC
:10177200AA81AD3531F4A98DA13018F0E98DE1507F
:10178200E98FAA81AE3559F4AF81B8850E949920BC
:1017920030F4EF81F885E456F040EF83F887AA81B0
:1017A200AF3531F4A88DA13018F0E88DE150E88F03
:1017B200AA81A03631F4AF89A13018F0EF89E15047
:1017C200EF8BAA81A13649F4A0911203A13028F02F
:1017D200E0911203E150E0931203AA81A23649F488
:1017E200A0910F03AB3028F0E0910F03EA50E09391
:1017F2000F03AA81A33649F4A0910E03A13028F069
:10180200E0910E03EA50E0930E0322FC26C0E09121
:101812001F03A4E9B3E0FF27662777270E94BC1DB8
:101822000E945320A0919403B09195038091960356
:10183200909197030E949D203CF40E94EF1A0E940F
:10184200F81A0E94FF1A09C0E0E0E0938403E093D3
:101852008503E0938603E093870322FE0CC0AA85EA
:10186200B0E00E94FA19A4E9B3E00E9465180E9450
:10187200EF1A0E94FF1A0E94EF1AACE1B3E00E9435
:10188200831DEC93A0912003B0E0E0E0F1E00E9420
:10189200C11FDF01E0912103F0E0EA0FFB1FA4E684
:1018A200B3E00E9465180E94081BA0E0B0E080E14E
:1018B20092E40E94941E7F936F93FF93EF930E9492
:1018C200E51A0E94111BAF91BF918F919F916627DC
:1018D20077270E94BC1D0E94461EE0936403F0938A
:1018E200650360936603709367030E94161BE0E032
:1018F200F0E060E87FE30E94FF1E0E2E0E94161B9E
:10190200E0E0F0E068E472E40E94F91EE021F9F000
:101912000E94081B0E94F81AA8E5B3E00E94851DE8
:101922000E9453200E94081BE0936803F09369030E
:1019320060936A0370936B030E94161B0E946F17D9
:101942000E94461EAEE2B3E00E948C1715C0E0E092
:10195200E0935803E0935903E0935A03E0935B0347
:10196200E0936803E0936903E0936A03E0936B03F7
:10197200E0932E03E0932F03A0918803B091890393
:1019820080918A0390918B030E9427180E94FF1E68
:10199200EF930E94A8170E94FF1EAF91EA2309F459
:1019A2003EC0E0911D03F0E0FF93EF930E949F176A
:1019B200E0E0F0E068EC72E40E94941EAF91BF9107
:1019C2000E94401F0E945A200E94BB170E941F1BA8
:1019D200A0916003B09161038091620390916303CF
:1019E200E0E0F0E064E172E40E94461EDF01CB0118
:1019F2000E94E7170E94941EA0E0B0E080E291E40A
:101A02000E94461E0E941F1BE0916003F091610339
:101A12006091620370916303DE010E94C0170E940D
:101A22005A19A0911003EDEF0E94591F0E220E9435
:101A32006019E02129F0E0911003EF5FE0931003B9
:101A4200A92DEAE00E945E1F0E2EA0911003EFEF77
:101A52000E94591F0E220E946019E02129F0E89489
:101A6200F0F8E0E0E0931003A0911003EEE10E9491
:101A7200451F0E2E0E946019E02119F0E1E0E0936B
:101A82001303E0911203E03019F4E0E0E093130352
:101A92000E941E180E9427180E948B1F0E94041A7F
:101AA200A09113030E946C1919F0E1E0E093130373
:101AB200A0911303AC3309F41FEF4420C9F4E02FC3
:101AC200F0E034960E944917AE0FBF1FE12F0E942B
:101AD200281BA4E00E943A17A02F0E94321BA0915B
:101AE20022030E943A17A12F0E943A170E94371B25
:101AF200E1E0E41509F057C04424A0910A030E94D2
:101B0200401BE0930B03F0E0BC96DF01E09107037A
:101B1200F0E0AE0FBF1FE0910803F0E0AE0FBF1F71
:101B2200E0910903F0E0AE0FBF1FE0910C03F0E07B
:101B3200AE0FBF1FEC89F0E0AE0FBF1FED89F0E0E2
:101B4200AE0FBF1FEE89F0E0AE0FBF1FE0910D0395
:101B52000E94281BACE20E943A17A09107030E9440
:101B62003A17A09108030E943A17A09109030E9414
:101B72003A17A0910B030E943A17A0910C030E94FE
:101B82003A17AC890E943A17AD890E943A17AE897A
:101B92000E943A17A0910D030E94321BA0E00E94FE
:101BA200321B0E94371B233608F000C3A0E0F799CE
:101BB200A1E0EA2FE295E07F0E2EA0E0F399A1E0EA
:101BC200EA2FEE0FEE0F0E0EA0E0F499A1E0EA2F3D
:101BD200EE0FA02DAE0FE0E0F599E1E0EA0FEB8FFA
:101BE200EAE0E8ABE9ABEAABEBABECABEDABEEAB0F
:101BF2000E94461BEAE0EAAFEBAFECAFEDAFEEAF0F
:101C02000E944B1BAA34E1E0BE07E0E08E07E0E051
:101C12009E071CF4E1E0E09302030E944B1BE9E4FF
:101C2200F1E060E070E00E94541BEEE5F1E060E05C
:101C320070E00E94831FE02119F0E3E0E0930203C9
:101C42000E944B1BEDE5F1E060E070E00E94541B46
:101C5200E8E6F1E060E070E00E94831FE02119F005
:101C6200E7E0E09302030E944B1BE7E6F1E060E04D
:101C720070E00E94541BECE7F1E060E070E00E942B
:101C8200831FE02119F0EFE0E09302030E944B1B57
:101C9200AC37E1E0BE07E0E08E07E0E09E071CF013
:101CA200EFE1E09302030E941E18AA30E0E0BE07B3
:101CB200E0E08E07E0E09E072CF00E941E180E94D2
:101CC200571BEAAB0E941E180E94601BEBABA0914F
:101CD2001C03AA3030F0B0E00E94FA190E94641B83
:101CE200E8AB0E946A1BE9AB0E94721B0E947C1B3C
:101CF2000E947F1BEEAB203079F5EFEAED8F0E9458
:101D0200821BA436E0E0BE0720F00E94821B0E94E4
:101D1200871B0E94821B0E94111B0E94921BEDAF27
:101D22000E94821B0E94981BA0910103AA3010F00E
:101D3200E2E0EFABA09101030E949E1BE8AFA091ED
:101D42000003B0E00E94FA190E94641BE9AFA0915F
:101D520000030E949E1BEAAF213099F5E89420F817
:101D6200EFE4ED8F0E941418A031E7E2BE0728F0DD
:101D72000E9414180E94A41BEAAF0E941418A83EE5
:101D8200E3E0BE0728F00E9414180E94A91BEBAFE3
:101D92000E941418A436E0E0BE0720F00E94141836
:101DA2000E94871B0E9414181A9738F00E94141878
:101DB2000E94111B0E94921BEDAF0E9414180E94F8
:101DC200981B223009F069C0E89420F8EFE0ED8F0B
:101DD200E7E7E8AFE4E7E9AFA0914D03AA2352F4A5
:101DE200E0914C03F0914D030E940F1FE0934C03CE
:101DF200F0934D030E94A8170E94BB17772312F499
:101E0200E0E4EDAF0E94A8170E94BB170E94AE1B30
:101E120010F4E0E4ECAF0E94A8170E94BB170E94E6
:101E2200B71B10F4E0E4EBAF0E94A8170E94BB17A7
:101E32000E94C01B10F4E0E4EAAF0E94C91BA0316B
:101E4200E7E2BE072CF00E94C91B0E94CE1BEAAF3C
:101E52000E94C91BA83EE3E0BE072CF00E94C91BEA
:101E62000E94D31BEBAF0E94C91BA436E0E0BE0761
:101E72002CF00E94C91B0E94D81BECAF0E94C91B08
:101E82001A973CF00E94C91B0E94FA190E94641B17
:101E9200EDAF0E94C91B0E94DD1B233009F05BC01D
:101EA2000E94E31BA0914F03AA2352F4E0914E0338
:101EB200F0914F030E940F1FE0934E03F0934F03E4
:101EC2000E94EC1B772312F4E0E4EDAF0E94EC1BBE
:101ED2000E94AE1B10F4E0E4ECAF0E94EC1B0E94E7
:101EE200B71B10F4E0E4EBAF0E94EC1B0E94C01B96
:101EF20010F4E0E4EAAF0E94F01BA031E7E2BE0773
:101F02002CF00E94F01B0E94CE1BEAAF0E94F01B35
:101F1200A83EE3E0BE072CF00E94F01B0E94D31BF8
:101F2200EBAF0E94F01BA436E0E0BE072CF00E944B
:101F3200F01B0E94D81BECAF0E94F01B1A973CF0DA
:101F42000E94F01B0E94FA190E94641BEDAF0E94CE
:101F5200F01B0E94DD1B2430C9F40E94E31BE0E564
:101F6200EAAFA0911B03A43620F0B0E00E94D81B78
:101F7200ECAFA0911B03B0E00E94FA190E94641B0F
:101F8200EDAFA0911B030E949E1BEEAF253039F5E9
:101F9200E89420F8EFE8ED8FE0E0E8AFE5E0E9AFA4
:101FA200E8E7EAAFA881B981A83EE3E0BE071CF0EA
:101FB2000E94D31BEBAFA881B981A436E0E0BE0733
:101FC2001CF00E94D81BECAFA881B9810E94FA19BB
:101FD2000E94641BEDAFA881B9810E94DD1B2630EF
:101FE200E9F5E89420F8EFE0ED8F1130C0F0ECE075
:101FF200E8AFA12F0E94401BE436A0E0FA0724F0CC
:10200200A12F0E94F51BE9AFA12F0E94401B3A9716
:1020120024F0A12F0E94FB1BEAAFA12F17C0EBE017
:10202200E8AFAA8D0E94401BE436A0E0FA0724F034
:10203200AA8D0E94F51BE9AFAA8D0E94401B3A9718
:1020420024F0AA8D0E94FB1BEAAFAA8DB0E0E2E069
:10205200F0E00E94DE1F0E94641BEBAF273009F004
:1020620071C0A0914803B0914903A135EBEFBE07BF
:1020720034F4E1E5FBEFE0934803F0934903A091C8
:102082004803B0914903A03BE4E0BE0734F0EFEA15
:10209200F4E0E0934803F0934903A0914903AA2393
:1020A2004AF4E0E4EBAFE0914803F09149030E9467
:1020B2000F1F04C0E0914803F0914903E0934A03E3
:1020C200F0934B03A0914A03B0914B03ECE3F0E091
:1020D2000E94DE1FE0933603F09337030E94011C37
:1020E200ECE30E94BB1FA0914A03B0914B03AE1BCD
:1020F200BF0BA0933803B0933903EFE2ED8F23FEB9
:102102001BC00E94011C1A9710F0E2E0EFAB0E9484
:10211200011C0E94061CE8AFA0913803B09139035C
:102122000E94111B0E94921BE9AFA0913803B0914B
:1021320039030E94061CEAAFE3E7ECAFE8E3EDAF38
:10214200E4E5EEAF0E940B1CAE2FE0911E030E944D
:10215200111CEA0F0E94171C0E94201CEC8FA985FB
:10216200A130D0F00E94461BE9E7EAAFE0E5EBAF11
:10217200ECAFA985B0E00E94FA190E94641BEDAF92
:10218200A9850E949E1BEEAF0E940B1C0E94171C89
:10219200E00DEC8FEFE0ED8FF29B08C00E940B1C6C
:1021A2000E94171C0E94201CEF5FEC8F233609F05F
:1021B20071C351E0503130F40E94291CEAE0EC93E3
:1021C2005F5FF8CFAA81ECE50E94301CEBE50E942C
:1021D200451FE02911F0EEE1EA83AA81AF3111F443
:1021E200EDE5EA83EA81E03029F4E0910703F0E0CB
:1021F200ED83FE83AA81A13029F4E0910803F0E087
:10220200ED83FE83AA81A23029F4E0910903F0E074
:10221200ED83FE83AA81A33029F4E0910A03F0E062
:10222200ED83FE83AA81A43029F4E0910C03F0E04F
:10223200ED83FE83AA81A53021F4EC89F0E0ED83E1
:10224200FE83AA81A63021F4ED89F0E0ED83FE83BE
:10225200AA81A73021F4EE89F0E0ED83FE83AA8102
:10226200A83029F4E0910D03F0E0ED83FE83AA810A
:10227200A93019F4E0E0ED83EE83AA81AA3019F4C3
:10228200E0E0ED83EE83AA81AB3019F4E0E0ED8368
:10229200EE83AA81AC3021F4E4E2F0E0ED83FE8328
:1022A200AA81AD3021F40E948B18ED83FE83AA81AE
:1022B200AE3021F4E889F0E0ED83FE83AA81AF30ED
:1022C20021F4E989F0E0ED83FE83AA81A03121F4B3
:1022D200EA89F0E0ED83FE83AA81A13121F4EC8545
:1022E200F0E0ED83FE83AA81A23121F4ED85F0E0D6
:1022F200ED83FE83AA81A33121F4EE85F0E0ED8324
:10230200FE83AA81A43121F40E94FF19ED83FE838A
:10231200AA81A53121F4EB81FC81ED83FE83AA81A0
:10232200A63129F4E0911703F0E0ED83FE83AA8140
:10233200A73129F4E0911903F0E0ED83FE83AA812D
:10234200A83129F4E0911803F0E0ED83FE83AA811D
:10235200A93121F4E32FF0E0ED83FE83AA81AA31B3
:1023620021F40E94EA1AED83FE83AA81AB3129F49B
:10237200E0911D03F0E0ED83FE83AA81AC3131F4DC
:10238200E0E022FCE1E0F0E0ED83FE83AA81AD31E2
:1023920021F40E945517ED83FE83AA81AE3121F408
:1023A2000E946117ED83FE83AA81AD3521F4E98D88
:1023B200F0E0ED83FE83AA81AE3521F4EF81F8854A
:1023C200ED83FE83AA81AF3521F4E88DF0E0ED8341
:1023D200FE83AA81A03621F4EF89F0E0ED83FE832B
:1023E200AA81A13629F4E0911203F0E0ED83FE8385
:1023F200AA81A23629F4E0910F03F0E0ED83FE8377
:10240200AA81A33629F4E0910E03F0E0ED83FE8366
:10241200AA81E0E00E94301CE3E00E94351CE1E169
:102422000E94351CE2E10E94351CE3E10E94351C4A
:10243200E5E10E94351CEBE10E94351CEDE10E94B2
:10244200451FE02911F0F69A01C0F698A0E0F6992E
:10245200A1E0EA2FE795E0E0E795ED8FE0E0EC8F71
:10246200EB8FE0930203AA81B0E0A7FDBFEF0E94C9
:10247200FA190E94641BEAABAA81B0E0A7FDBFEF84
:10248200EAE0F0E00E941020EBABAD81BE81A0310A
:10249200E7E2BE0718F00E94A41BEAAFAD81BE813D
:1024A200A83EE3E0BE0718F00E94A91BEBAFAD8186
:1024B200BE81A436E0E0BE0710F00E94871BAD810A
:1024C200BE811A9728F00E943A1C0E94921BEDAF1F
:1024D200AD81BE810E94981BAA81E1E10E94301C5D
:1024E200E2E10E94351CE3E10E94351CE5E10E9415
:1024F200351CEDE10E94451FE02929F00E943A1C9B
:102502000E94921BEDAFE7EAE0937A00A7E00E94F7
:1025120076180E949718E7E2E0937A00AA810E9457
:10252200B218AA81EEE00E94351CE1E10E94451F2B
:10253200E02911F0E1E06E2EAA810E94B718AA816B
:10254200EFE00E94351CE2E10E94451FE02911F0F4
:10255200E2E06E2EAA81E7E00E94301CE0E10E94D8
:10256200351C0E943D1C11F0E3E06E2E0E944917BB
:10257200D39708F452C00E94CB180E94D018E62DBF
:102582000E94D71820F0E8ECF0E00E949718E62DA0
:102592000E94E7180E94421CAC91A130E8F10E940F
:1025A200491C0E9407190E94A8204CF40E94421C58
:1025B2000E94521C0E94051F0E945D1C23C00E94A3
:1025C200661C0E942919EF930E94661C0E94321910
:1025D200AF91EA2379F00E94421C0E94521C0E9491
:1025E2000A1FA0935403B09355038093560390930C
:1025F200570308C00E94661C0E943B191CF00E94EF
:10260200681C0AC0A0915403B091550380915603EF
:10261200909157030E944D1904C00E9454190E94C0
:10262200681CAA81AD3049F40E94721B0E947C1B77
:102632000E947F1BEEABE0E2EB8FAA81A53149F449
:102642000E94721B0E947C1B0E947F1BEEABE0E685
:10265200EB8FAA810E94B218AA81EEE00E94351C7B
:10266200E1E10E94451FE029A9F00E94701CE4E00C
:102672000E94741C18F00E947A1CECAB0E9449174D
:102682001A9728F00E94801C0E94921BEDAB0E94B8
:10269200821CEEABAA810E94B718AA81EFE00E94C9
:1026A200351CE2E10E94451FE029A9F00E94701C3E
:1026B200E2E00E94741C18F00E947A1CECAB0E94AB
:1026C20049171A9728F00E94801C0E94921BEDABBA
:1026D2000E94821CEEABAA81E7E00E94301CE0E17E
:1026E2000E94351C0E943D1CA9F00E94701CE1E072
:1026F2000E94741C18F00E947A1CECAB0E944917CD
:102702001A9728F00E94801C0E94921BEDAB0E9437
:10271200821CEEABAA81A63121F40E94841CEBE05C
:10272200EBAFAA81A73121F40E94841CE0E4EBAF55
:10273200AA81A83121F40E94841CECE0EBAFAA81AB
:10274200A93169F4A0911C03B0E00E94FA190E9419
:10275200641BECAB0E946A1BEDABE7E7EEABAA8110
:10276200AA31A9F40E948B1CE4E6F0E00E94CB1F80
:102772000E94921BECAB0E948B1C0E94111B0E94B8
:10278200921BEDAB0E948B1C0E94061CEEABAA8131
:10279200AB3159F4ECE7E8AFE7E7E9AFE8E7EAAFD6
:1027A2000E943A1C0E94921BEDAFAA81EDE10E94A9
:1027B200301CEEE10E94451FE029D9F0E3E7E8AFC3
:1027C200E8E3E9AFAA81AD3111F4EEE501C0E8E733
:1027D200EAAF0E94901C1A9738F00E94901C0E9447
:1027E200111B0E94921BEDAB0E94901C0E94061CC2
:1027F200EEABAA81E1E10E94301CE2E10E94351CAD
:102802000E943D1C11F0E8E7E9AFAA81AD3541F520
:10281200E7E7EBAFEEE5ECAFE9E3EDAFE98DEEAF65
:10282200E7EAE0937A00A98D0E9476187E2EE7E20D
:10283200E0937A00E3E6E71528F4A72DB0E00E94C2
:10284200D81BECABE9E0E71538F4A72DB0E00E9405
:10285200FA190E94641BEDABA72D0E949E1BEEABE2
:10286200AA81AE3521F4EEE5E8AFE1E0E9AFAA8155
:10287200AF3521F4EEE5E8AFE2E0E9AFAA81A03698
:1028820021F4EEE5E8AFE3E0E9AFAA81A23611F464
:10289200E0E1EB8F51E0503108F077C00E94291C33
:1028A200EC91E03021F40E94291CEFE3EC930E94AA
:1028B200291CAC91A63021F40E94291CEDE7EC936F
:1028C2000E94291CAC91A13021F40E94291CE6E04F
:1028D200EC930E94291CAC91A23021F40E94291C85
:1028E200EBE5EC930E94291CAC91A33021F40E94E9
:1028F200291CEFE4EC930E94291CAC91A43021F432
:102902000E94291CE6E6EC930E94291CAC91A5309A
:1029120021F40E94291CEDE6EC930E94291CAC9143
:10292200A73021F40E94291CE7E0EC930E94291CA5
:10293200AC91A83021F40E94291CEFE7EC930E948D
:10294200291CAC91A93021F40E94291CEFE6EC93DA
:102952000E94291CAC91AA3021F40E94291CE0E0BB
:10296200EC930E94291CAC91AB3021F40E94291CEB
:10297200E1E0EC930E94291CAC91AC3021F40E945E
:10298200291CE8E0EC935F5F86CFE0910203E695B5
:10299200E6950E94951CECA90E949B1CECA90E9442
:1029A200A61CECA90E94B11CECA90E94B81CECA9BF
:1029B2000E94BF1CECA90E94C61CECA90E94CD1C5F
:1029C200EF8FE0910203E695E695E6950E94951C4D
:1029D200EDA90E949B1CEDA90E94A61CEDA90E94D4
:1029E200B11CEEA90E94B81CEEA90E94BF1CEEA960
:1029F2000E94C61CEEA90E94CD1CE8A3E09102032E
:102A0200E6950E94951CEEA90E949B1CEEA90E94CD
:102A1200A61CEEA90E94B11CEDA90E94B81CEDA94A
:102A22000E94BF1CEDA90E94C61CEDA90E94CD1CEC
:102A3200E9A3EFA90E94951CE8AD0E949B1CE8AD9A
:102A42000E94A61CE8AD0E94B11CED8D0E94B81C2C
:102A5200ED8D0E94BF1CED8D0E94C61CE091020309
:102A6200E170EA2BEAA3ECAD0E94951CECAD0E944A
:102A7200D31CECAD0E94DC1CECAD0E94E51C0E9454
:102A8200EF1CECAD0E94F31CECAD0E94FC1CECAD03
:102A9200E295E170EA2BEBA3EBAD0E94951CEBAD46
:102AA2000E94D31CEBAD0E94DC1CEBAD0E94E51C26
:102AB200E2950E94B81CEDAD0E94F31CEDAD0E94A0
:102AC200FC1CEDADE295E170EA2BECA3ED8D0E94CA
:102AD200051DEBAD0E949B1CEBAD0E94A61CEBAD4D
:102AE2000E94B11CEAAD0E94B81CEAAD0E94BF1C54
:102AF200EAAD0E94C61CEAAD0E94CD1CEDA3EDAD6D
:102B02000E94951CEDAD0E94D31CEDAD0E94DC1C11
:102B1200EDAD0E94E51C0E94091D0E94B81CEAADA1
:102B22000E94F31CEAAD0E94FC1CEAADE295E17042
:102B3200EA2BEEA3E9AD0E94951CE9AD0E94D31CDD
:102B4200E9AD0E94DC1CE9AD0E94E51CEE1FE0E04D
:102B5200EE1F0E94B81CEEAD0E94F31CEEAD0E9467
:102B6200FC1CEEADE295E170EA2BEFA3EC8DE29551
:102B72000E94951CE9AD0E949B1CE9AD0E94A61C17
:102B8200E9AD0E94B11CE8AD0E94B81CE8AD0E94FC
:102B9200BF1CE8AD0E94C61CE8AD0E94CD1CE8A790
:102BA200EEAD0E94951CEEAD0E94D31CEEAD0E94CC
:102BB200DC1CEEADE695E695E6950E940E1DE8A9B1
:102BC200EE1FE0E0EE1F0E94B81CE8A9E295E1705A
:102BD200EE0FEE0FEA2BAE2FE8A90E94FC1CE8A92B
:102BE200E295EF70E695E170EA2BE9A7E8A9E69590
:102BF200E695E6950E94951CE8A9E695E6950E9461
:102C0200141DE8A90E941C1DE8A90E940E1DEC8D4E
:102C12000E94EF1CEC8D0E94111CEA2BAE2FEC8D52
:102C22000E94241DEC8DE695E170EA2BEAA7EC8D5B
:102C32000E94051DE9A9E2950E94141DE9A90E94BE
:102C4200A61CE9A90E94291DE9A90E94EF1CE9A975
:102C52000E94111CEA2BAE2FE9A9E6950E94241DC1
:102C6200E9A9E170EA2BEBA7EC8D0E94091D0E94F5
:102C7200951CEB8D0E94141DEB8D0E941C1DEB8D8B
:102C8200E695E6950E940E1DE0910203E2950E94F0
:102C9200B81CEC8DEE1FE0E0EE1FE170EE0FEE0FC0
:102CA200EA2BAE2FEB8DE695E695E6950E94241D64
:102CB200EB8DE295E170EA2BECA7EB8D0E94051DEE
:102CC200EAA9E2950E94141DEAA90E94A61CEAA99B
:102CD2000E94291DEBA90E94EF1CEBA90E94111C66
:102CE200EA2BAE2FEBA9E6950E94241DEBA9E17019
:102CF200EA2BEDA7EB8D0E94091D0E94951CEBA902
:102D0200E2950E94141DEBA90E94A61CEBA90E9449
:102D1200291DEAA90E94EF1CEAA90E94111CEA2BB4
:102D2200AE2FEAA9E6950E94241DEAA9E170EA2BDA
:102D3200EEA70E942D1D5D3078F40E94331DA2E59E
:102D4200B8E00E94231FE17011F45D9801C05D9A02
:102D52000E943A1D5F5FEFCF0E94421D5D3078F402
:102D62000E94331DA0E3B8E00E94231FE17011F41A
:102D72005D9801C05D9A0E943A1D5F5FEFCF0E948D
:102D8200421D5D3078F40E94331DA2E0B8E00E943B
:102D9200231FE17011F45D9801C05D9A0E943A1DF3
:102DA2005F5FEFCF0E94421D5D3078F40E94331DB9
:102DB200A6E0B8E00E94231FE17011F45D9801C003
:102DC2005D9A0E943A1D5F5FEFCF0E94421D5A300A
:102DD20098F45E9885E28A95F1F7E9E0E51BA0E4B4
:102DE200B1E00E94231FE17011F45D9801C05D9A69
:102DF2000E943A1D5F5FEBCF41E04131E8F451E0C0
:102E02005930C0F45E9885E28A95F1F7E42FF0E03C
:102E1200DE015E96AE0FBF1FAC91E8E0E51B0E949B
:102E22001B1FE17011F45D9801C05D9A0E943A1D6A
:102E32005F5FE6CF4F5FE1CF5D9A85E28A95F1F75A
:102E4200289A8DEC9AE00197F1F7AB2DE4E60E9407
:102E52005E1F0E2EA0E0F099A1E00E94781929F0E1
:102E6200A4E6B0E00E944C1DF09A0C948404EF9604
:102E7200FFCFAA93E091C000E072E1F3E881E09312
:102E8200C60021960895A0912603B09127030895C4
:102E9200A0912203B09123030895E0E0F0E061EEF7
:102EA20075E40E94941E0895E0913403F091350375
:102EB2000895662777270E94BC1D0E94532008951B
:102EC200E0914003F09141030895A0917003B09105
:102ED200710380917203909173030895E0E0F0E032
:102EE20060E271E40895A0913403B091350308952E
:102EF200E0E0F0E00E94751F0895A0914003B091B8
:102F020041030895E0919803F091990360919A0327
:102F120070919B0308950E94831DED93FC93089585
:102F2200A0918403B09185038091860390918703D9
:102F320008950E94461EDF01CB01AFCFA09180030E
:102F4200B091810380918203909183030895A091AF
:102F52001D03E4E6EA9FF001DF01E0918003F091B6
:102F6200810360918203709183030E94401F0E943B
:102F72005A2008950E945D200E94EF1D08950E942C
:102F8200851DED93FC930895E0915C03F0915D0340
:102F920060915E0370915F030895EA9FF001DF0183
:102FA200E091A003F091A1036091A2037091A303A9
:102FB2000E94401F0E945A20DDCFE0918C03F091C5
:102FC2008D0360918E0370918F030895E0918803C1
:102FD200F091890360918A0370918B030895A09107
:102FE2006C03B0916D0380916E0390916F0308950D
:102FF200E0936C03F0936D0360936E0370936F0321
:103002000895A0917403B091750380917603909115
:1030120077030895E0916C03F0916D0360916E0364
:1030220070916F030895A0912A03B0912B03089524
:10303200E0E00E945E1F0E2E0895A0915803B09109
:10304200590380915A0390915B030895E0E0F0E008
:1030520060E070E008950E22A0911303ECE30E9459
:10306200591FE0210895A0913C03B0913D0340CF48
:10307200A4E1B0E00E944C1DE7EAE0937A000895D3
:10308200A4E00E94FA02EF2FF0E09E2EE7E2E09326
:103092007A000895EBE0E093A903E8EBE093AA033A
:1030A2000895E8ECF0E0E0934403F09345030895BB
:1030B200E0EDF7E0E0934603F09347030895E093D1
:1030C2002C03F0932D0308950E943B1F0E94BC1D08
:1030D2000E9453200895E0933203F093330308953E
:1030E200E0933C03F0933D0308950E94FA02EF2F10
:1030F200F0E008950E94FA020E94301F0E942C1FE5
:103102000895E0935C03F0935D0360935E03709314
:103112005F030895E0912C03F0912D030895E7E2F7
:10312200E0937A00E7EAE0937A000895E0932203BD
:10313200F09323030895ACDEEAEFF0E00895A8DEF1
:10314200EEE1F0E00E946F1F08950E2EA52DE1E042
:103152000E945E1F0E22A985E5E00E94591FE02110
:103162000895E5E00E94451F0E2E0895E6E00E94B4
:10317200451F0E2E0895AD2DEAE00E94591F0E2E16
:10318200A0E0F3FCA1E0E0E00E94451F0E22A22F86
:10319200E3E60895E0912203F09123030895F29764
:1031A200ADE7B0E00E94931F0F010895F0E0DE0149
:1031B2001F96AE0FBF1FEC91F0E0D0010E94CB1F13
:1031C200B5DF66DEA93CE0E0BE070895F0E0DE016F
:1031D2005396AE0FBF1FEC91F0E05ADE0E94931F90
:1031E200DF01E4E6F0E00E94CB1FA0CFE02FF0E089
:1031F200DE011B96AE0FBF1F0895A0915003B09140
:10320200510380915203909153030895E8EEF3E045
:1032120060E070E00E940820DF01CB01BBDF66277F
:1032220077270895EC91F0E00E943B1FA8E0BCE4F0
:1032320081E090E00E940820E0CFE0935003F093F9
:10324200510360935203709353030895D6DFDECF88
:103252000E940A1FE5E0F0E060E070E00E948B1F30
:1032620008950E940A1FE4E1F0E060E070E00E942D
:10327200831F08950E940A1FA431E0E0BE07E0E028
:103282008E07E0E09E070895EF81F885D6DE662777
:1032920077270E94C61FD1CFE8EEF3E060E070E02E
:1032A2000E94082043CFE0E0E0932203E09323034F
:1032B2000895A92DEAE00E94591F0E2E0895A22F0B
:1032C200E3E60E94591F0895A0E0F0FCA1E0E0E0CF
:1032D2000E94451F0895E0E00E945E1FE0210895CC
:1032E200E0911903AADEFF27662777270895E0E019
:1032F2000E94451FE0210895EB81FC81A0915C03AF
:10330200B0915D0380915E0390915F0366277727FA
:1033120008950E2EA0915C03B0915D0380915E032F
:1033220090915F030895EAE0F0E060E070E00895B4
:103332002BDEAB81BC81882799270E940A1F089542
:10334200A630E0E0BE07E0E08E07E0E09E070895C9
:10335200A0914403B09145030895E0914403F09194
:1033620045030895E0934403F09345030895E32F42
:10337200A0919403B0919503809196039091970345
:10338200FF27662777270E94BC1D0E94D91E089539
:10339200E32FF0E0A0919403B091950380919603FE
:1033A200909197030E943B1F0E94BC1DE3CDA09108
:1033B2004603B09147030E94401F0E945A20DACD73
:1033C200E0934603F09347030895A32FBB27E091B0
:1033D2009403F091950360919603709197030E9474
:1033E200401F0E945A20C6CDE0914603F091470348
:1033F2000895EAE0F0E00E94DE1F0895E0913C03A8
:10340200F0913D0308950E2EA0911303ECE30E9468
:10341200591F0E220895E0910803A0E0B0E00E9437
:103422008220E0910903A1E0B0E00E948220E091B5
:103432000A03A2E0B0E00E948220E0910C03A3E024
:10344200B0E00E948220EC89A4E0B0E00E948220D9
:10345200ED89A5E0B0E00E948220EE89A6E0B0E00E
:103462000E948220E0910D03A7E0B0E00E9482203A
:10347200E0910E03A8E0B0E00E948220E0910F03E9
:10348200A9E0B0E00E948220E0911203AAE0B0E03D
:103492000E9482203FDEA9E1B0E00E947A20E88902
:1034A200A4E1B0E00E948220E989A5E1B0E00E9497
:1034B2008220EA89A6E1B0E00E948220EC85ABE09E
:1034C200B0E00E948220ED85ACE0B0E008950E9459
:1034D2008220EE85ADE0B0E00E948220EB81FC818B
:1034E200AFE1B0E00E947A20E0911703AEE0B0E0D5
:1034F2000E948220E0911903AFE0B0E00E94822096
:10350200E0911803A0E1B0E00E948220E32FA1E144
:10351200B0E00E948220EF81F885A1E2B0E00E9433
:103522007A20E88DA2E1B0E00E948220EF89A3E137
:10353200B0E00E948220E0918003F09181036091CB
:10354200820370918303A3E2B0E00E94851D0E9472
:103552007A20E0913203F0913303A5E2B0E00E94B9
:103562007A20E0911D03A7E1B0E00E948220E0E012
:1035720022FCE1E0A8E1B0E00E9482203FDFA7E266
:10358200B0E00E947A2008950E94591F0E2EA0E0FA
:10359200F2FCA1E0E0E00E94451F0E220895A82D52
:1035A200EAE00E94591F0E2E0895A0E0F1FCA1E06E
:1035B200E0E00E94451F0E2208950E22A22FE3E6AC
:1035C2000E94451FE0210895A0913203B091330378
:1035D2000895E0913203F09133030895E09194034A
:1035E200F091950360919603709197030895A0E07E
:1035F200B0E080E09FE30E94F61D0895E09384030B
:10360200F093850360938603709387030895E09196
:103612006403F091650360916603709167030895F6
:10362200EAE0F0E00E94CB1F0895A0916403B091FC
:10363200650380916603909167030895E0936003A8
:10364200F093610360936203709363030895F0E063
:10365200EA0FFB1FE0933003F0933103AEE30C94C7
:103662003A170E943A17A0E00C943A17E0913103FE
:10367200AE2F0E943A17A09130030C943A17B0E093
:10368200E2E0F0E00E94DE1F0895EAE0EFABE8AF6F
:10369200E9AF0895A0915C03B0915D0380915E0350
:1036A20090915F0308950E948B1F33CE3CDE0E94EF
:1036B2000820DF01CB0137DE0E941E20089533DE91
:1036C2000E941E200895DF01EAE0F0E00E9410202F
:1036D2000895A0911C03BB27EAE0F0E00E941020AD
:1036E2000895D8DFE4E6F0E060E070E00E94082090
:1036F200DF01CB01E4CFECABCDDFD8CFEDABCADF3E
:10370200DECFA0912803B09129030895E4E6F0E00A
:103712000E94CB1FDF01EAE0F0E00E940D20ECAF37
:103722000895DF01EAE0F0E00E940D200895EAE04A
:10373200F0E00E940D20EEAF0895BB27EAE0F0E032
:103742000E9410200895E0E1F7E20E94CB1FE9CF2A
:10375200E8EEF3E00E94CB1FE4CFDF01CB01E0E013
:10376200F0E060E171EC0E94D91E0895DF01CB0107
:10377200E0E0F0E066EC72EC0E94D91E0895DF01F1
:10378200CB01E0E0F0EC69E774EC0E94D91E0895E9
:10379200A0914C03B0914D030895E0E1F7E20E943D
:1037A200DE1F91CFE8EEF3E00E94DE1F8CCFE4E64D
:1037B200F0E00E94DE1F87CFEAE0F0E00E941020D6
:1037C200EEAF0895E89420F8EFE8ED8FEEE3E8AF6E
:1037D200E4E7E9AF0895A0911D03E4E6DECBA091F2
:1037E2004E03B0914F030895B0E0E8ECF0E00E9480
:1037F200DE1F69CFB0E0E4E1F0E00E94DE1F63CF9C
:10380200A0913603B09137030895EAE0F0E00E94F8
:103812000D200895E0911E03E170EE0FE058089527
:10382200E695E695E170EE0FEE0F08950E2EA0E0FC
:10383200F199A1E0EA2FEE0FEE0FEE0F08950E0EB2
:10384200A0E020FCA1E0EA2FE295E07FE00D0895E0
:10385200E52FF0E0DE019F96AE0FBF1F08950E9494
:10386200451F0E2EAA8108950E94451F0E2AAA8185
:103872000895AD81BE81D4CEE3E10E94451FE029C7
:103882000895E62DF0E0DE011B96AE0FBF1F0895EE
:10389200A0915403B0915503809156039091570320
:1038A2000895EC91F0E00E943B1FA8E0BCE481E0A7
:1038B20090E00E940820ECCFE0935403F09355036C
:1038C20060935603709357030895E2DF9FCCEF8114
:1038D200F885B3DB662777270E94C61FEDCF5ADC37
:1038E200F695E79523CCEB8FD3DAA436E0E0BE075A
:1038F2000895CEDAE4E6F0E00E94CB1F12CFC8DAD8
:103902008FCEC6DA82CFE9E3E8AFE0E5E9AFEEE3D6
:10391200EAAF0895A0912E03B0912F030895A091CC
:103922003A03B0913B030895E170E795E0E0E79533
:10393200AE2F0895E295EF70E695E170E295E07F93
:10394200EE0FEE0FEA2BAE2F0895E295EF70E6959B
:10395200E695E170E295E07FEE0FEA2BAE2F089537
:10396200E295E170E295E07FEA2BAE2F0895E170D7
:10397200EE0FEE0FEE0FEA2BAE2F0895E695E170F3
:10398200EE0FEE0FEA2BAE2F0895E695E695E17065
:10399200EE0FEA2BAE2F0895E695E695E695E170D7
:1039A200EA2B0895E695E170E295E07FEE0FEE0FC7
:1039B200EA2BAE2F0895E695E695E170E295E07F59
:1039C200EE0FEA2BAE2F0895E695E695E695E170A7
:1039D200E295E07FEA2BAE2FED8D0895E695E69510
:1039E200E695C5CFE295EF70E695E170EE0FEE0F2A
:1039F200EA2BAE2F0895E295EF70E695E695E17019
:103A0200EE0FEA2BAE2F0895E295EF70E6958CCF7C
:103A1200E295EF70E695E6950895E170E295E07F14
:103A2200EA2BAE2F0895E170E295E07FEE0FEE0FE4
:103A3200EA2BAE2F0895E695E170E295E07FEE0F56
:103A4200EA2BAE2F0895E170EE0FEA2BAE2F089508
:103A5200E295EF70E695E1CF289885E28A95F1F735
:103A620051E008955E9885E28A95F1F7ECE0E51B56
:103A7200089585E28A95F1F75E9A85E28A95F1F7D3
:103A820008955D9A85E28A95F1F7289A84E191E09A
:103A92000197F1F7E1CF109639F08DEC9AE001979A
:103AA200F1F7A8951197C9F70895552342F45038B4
:103AB20011F4E0FF04C03196691F791F6BF050E8E2
:103AC200572711F45F93CFC05F3F31F0660F000CB0
:103AD20057956795752F08955F9300200AF0CFC020
:103AE200C8C050E8192E1522880F991F9527550F27
:103AF200879550E8072E0522660F771F7527550F09
:103B020067950895689401C0E8945F93F2DF703876
:103B120018F07F3F08F4A7C056E1571BAAF451954D
:103B220058300EF4593030F0EFEFFFEF6FEF7FE7D0
:103B320077F91AC077275523B9F0EE0FFF1F661FDA
:103B4200771F5A95D1F710C07727583028F0EF2FFA
:103B5200F62F672F5850F9CF552331F07695679598
:103B6200F795E7955A95D1F700200AF45BD15F915A
:103B72000895689401C0E894309760407040B1F0B5
:103B8200002426F0772312F400944CD1172E7EE104
:103B9200112032F07A95EE0FFF1F661F111CF9CF2C
:103BA200EF2FF62F612D5F938ADF5F9108954F9378
:103BB200AF01FD01DA01AB01BC01CA01402D012CAC
:103BC200142E4F910895EA0FFB1F681F0895E09588
:103BD200F0956095EF5FFF4F6F4F08955F9381DF20
:103BE200903871F150E8152604C05F937ADF90385F
:103BF20039F1703821F1572F591B2BF112F4D7DF0D
:103C0200FACF583118F0AA27BB278827583028F056
:103C1200AB2FB82F88275850F9CF552329F0869516
:103C2200B795A7955A95D9F7502D512572F0CBDF4C
:103C320038F46795F795E795739513F420C0B7DFCD
:103C42003EDF5F910895D8F7FBCFEA1BFB0B680BB1
:103C520051F010F40094BBDF662392F3EE0FFF1FC6
:103C6200661F7A95CBF7EE27FF27662777275F91A6
:103C72000895EFEFFFEF6FE77FEF5F910895EFEFAA
:103C8200FFEF6FE77FE75F9108955F932ADF703858
:103C920051F3903841F301240894791F23F41CF363
:103CA20000203AF3ECCF0F921F932F933F934F9341
:103CB200112722279927689FA0018F9F302D410D40
:103CC200591F6B9F300D411D591F8E9F27D0BF9FDB
:103CD20025D06A9F23D0BE9F1DD0AF9F1BD0AE9F21
:103CE200110D291F391F491F591FE32FF42F652F6B
:103CF200522F4F913F912F911F910F9066232AF0DF
:103D0200550FEE1FFF1F661F02C073954BF2CDDEEB
:103D12005F910895100D211D391F02C0200D311D24
:103D2200491F591F08955F93DCDE703821F411207A
:103D32000AF49FCFA4CF903809F495CF01240894B8
:103D4200970B1BF4D4F30020F3CF792F1F932F93FB
:103D52003F934F93112411272227332744275527B6
:103D620090E2AE17BF078607410730F0AE1BBF0BCC
:103D7200860B410B089401C08894551F221F331FE4
:103D8200111CAA1FBB1F881F441F9A9551F7F901E6
:103D9200612D4F913F912F911F91662332F0550F64
:103DA200EE1FFF1F661F7A9543F27FDE5F91089533
:103DB20099239AF0772342F0971748F029F4AE1727
:103DC200BF07860720F031F098948894089598945C
:103DD200089408951894889408957723C2F7971742
:103DE20098F3A9F7EA17FB07680788F399F3ECCF72
:103DF200DFDFE1E009F008F0EE270895D9DFE1E026
:103E020009F008F4EE270895EA0FFB1F681F791FD7
:103E12000895AE1BBF0B860B970B0895F195E195A4
:103E2200F0400895F09560957095E195FF4F6F4FC2
:103E32007F4F0895EE230E2EEA2F19F0E6950A948D
:103E4200E9F70895EE230E2EFD0121F0F695E79590
:103E52000A94E1F70895F695E795F695E795F695B4
:103E6200E795F695E7950895FE2FFF0FFF0B6F2F4D
:103E72007F2F08956F2F660F660B762F08958B2F75
:103E8200880F880B982F0895EA17E1E009F0EE27D2
:103E92000895AE17E1E00CF4EE270895AE17E1E0C5
:103EA2000CF0EE270895EA17E1E00CF0EE270895F2
:103EB200AE17E1E008F0EE270895EA17E1E008F016
:103EC200EE270895EA17FB07E1E009F0EE270895CF
:103ED200AE17BF07E1E008F4EE270895AE17BF075B
:103EE200E1E008F0EE270895EA17FB07E1E008F0A9
:103EF200EE270895EA17FB0768077907E1E009F062
:103F0200EE270895AE17BF0786079707E1E00CF08A
:103F1200EE270895EA17FB0768077907E1E00CF03E
:103F2200EE270895FA9FF02DEB9FF00DEA9FE02D0A
:103F3200F10D08957A9F702D6B9F700DF89F700D93
:103F4200E99F700D6A9F602D710DFB9F600D711DC1
:103F5200E89F600D711D8827FA9FF02D610D781F73
:103F6200EB9FF00D611D781FEA9FE02DF10D681F98
:103F7200781F08956E2F6A9FF0016B9FF00D0895D0
:103F820070D0D0DF0EF44ADF089579D0D3DF0EF47B
:103F920049DF08950024112490E1AA0FBB1F001CE1
:103FA200111C0E1A1F0A18F40E0E1F1E01C0A1606A
:103FB2009A9599F7FD01D001089553D0EBDF0EF4E5
:103FC2002DDF08953F934F935F93002411244427DC
:103FD200552730E2AA0FBB1F881F991F001C111C16
:103FE200441F551F0E1A1F0A460B570B28F40E0EBC
:103FF2001F1E461F571F01C0A1603A9559F7FD01C8
:10400200BC01D001CA015F914F913F91089537D011
:10401200D9DF0EF407DF0895BDDFFD010895E894AE
:10402200B7FF04C0A095B09511966894F7FDF6DE2F
:10403200B1DFFD010EF4F2DE0895E89497FF09C0A6
:10404200A095B09580959095AF5FBF4F8F4F9F4FD2
:10405200689477FDE7DEB6DFFD01BC010EF4E2DE17
:104062000895E894F7FF02C0D9DE6894B7FF06C04E
:10407200A095B095119600F8039400FA0895E8947B
:1040820077FF02C0CFDE689497FF0BC00024A09593
:10409200B095809590951196801D901D00F803941F
:1040A20000FA0895ED93FD936D937C9308956894BF
:1040B20001C0E89401D060DD182E862F612D192EE3
:1040C200972F712D1B2EBF2FF12D1A2EAE2FE12D02
:1040D2000895119602D0FE2F1197F999FECFFF9302
:1040E200FFB7F894A1BDB2BDF89AE0B5FFBFFF914A
:1040F200089507D01196EF93EF2F03D0EF91119708
:104102000895F99B02C0A895FCCF9FB7F894A1BD72
:10411200B2BDF89A80B5E81719F0E0BDFA9AF99A9B
:104122009FBF089500240E160F060606070608957F
:1041320000240A160B06089500240A160B06080628
:1041420009060895EA17FB07680779070895AE176D
:10415200BF07860797070895E894EE2309F068944D
:104162000895AC0FBD1F05900D928A95E1F7089551
:00000001FF
